:020000000F28C7
:10000800CE00030E83129000040891000A089200A3
:100018004F089300C62A9C2B103083168500860152
:100028008B1681160116811507308104FF30831263
:100038008100AF01B001B101B2018511B90103140A
:10004800B90DF122533037237430372372303723F8
:100058006F303723623037236F30372373303723BD
:100068006B303723C0301A236F3037237030372373
:10007800203037232D303723203037234B30372398
:1000880031303723353037234B2864004B28013073
:100098008312AF070318B00A0030B00730082F04E6
:1000A800031D5728582849285C285C2864005C28C8
:1000B80001308312AF070318B00A0030B0073008C8
:1000C8002F04031D682869285A286D286D286400A4
:1000D8006D2801308312AF070318B00A0030B0074B
:1000E80030082F04031D79287A286B287E287E285B
:1000F80064007E2801308312AF070318B00A00306D
:10010800B00730082F04031D8A288B287C288B17FA
:10011800640001308312AF070318B00A0030B0073B
:1001280001302F063004031D9A289B28CC28003064
:10013800AE000030AD000030AC000030AB00051A56
:10014800A628A728CC2880301A23BA280230831280
:10015800A2002208B90034303723C4288312B90119
:100168000314B90D32303723C428C4288312390840
:10017800013A0319AA28033A0319B228C428C42843
:100188008312051EC828C928C428CC28CC28CC2806
:100198000130B1070318B20A0030B2070130310646
:1001A8003204031DD828D9288C282E08AA002D0827
:1001B800A9002C08A8002B08A7002A0897002908DE
:1001C8009600280895002708940000309B0093307B
:1001D8009A00E430990082309800AF218312170802
:1001E800AA001608A9001508A8001408A7003908CD
:1001F800A200A301A401A5012508970024089600E0
:1002080023089500220894002A089B0029089A00D0
:1002180028089900270898007B2283121708AA004B
:100228001608A9001508A8001408A7003930A2006C
:100238002208A6001F2900309700003096000030E1
:1002480095000A3094002A089B0029089A0028087B
:100258009900270898001E2283121408303EA20035
:100268000130A6022608840022088313800000308B
:10027800970000309600003095000A3094002A0854
:100288009B0029089A002808990027089800AF21A0
:1002980083121708AA001608A9001508A800140850
:1002A800A7002A08290428042704031D5C295D29BE
:1002B8001F29692969292030A2000130A6022608D1
:1002C800840022088313800069293330A20026089D
:1002D8002202031C702971295F29722980301A2390
:1002E8007C293430372385293230372385298529DD
:1002F80083123908013A03197829033A0319752931
:1003080085292D30372354303723203037232030A8
:1003180037232030372383123308372383123408D6
:100328003723C0301A23831235083723831236083F
:1003380037238312370837238312380837232030AE
:10034800372372303723703037236D3037238C28AA
:100358008C288C280F2800308312A00000309F00C2
:1003680000309E0000309D00170816041504140480
:100378000319BF29C029142AA1010314A10DD229E8
:1003880001309C000310940D950D960D970D9C0B54
:10039800C62901309C001C08A107D229971FD5291E
:1003A800D629C429D829D82901309C0003109D0DCD
:1003B8009E0D9F0DA00D9C0BDA2917081B02031D2B
:1003C800EF2916081A02031DEF2915081902031D43
:1003D800EF2914081802031CF229F329032A140828
:1003E80098021508031C150F99021608031C160F0E
:1003F8009A021708031C170F9B021D14032A0130C9
:100408000310970C960C950C940CFF3E031D042AC0
:100418000130A102031D112A122AD829142A142AEC
:10042800200897001F0896001E0895001D089400D4
:100438001D2A08008312170816041504140403194A
:10044800262A272A712A9D0103149D0D392A013075
:100458009C000310940D950D960D970D9C0B2D2A5D
:1004680001309C001C089D07392A971F3C2A3D2A09
:100478002B2A3F2A3F2A17081B02031D4D2A16085C
:100488001A02031D4D2A15081902031D4D2A1408C6
:100498001802031C502A512A602A140898021508C9
:1004A800031C150F99021608031C160F9A02170849
:1004B800031C170F9B02602A01300310970C960C3F
:1004C800950C940CFF3E031D612A01309D02031D0B
:1004D8006E2A6F2A3F2A712A712A1B0897001A0868
:1004E800960019089500180894007A2A0800003028
:1004F8008312A00000309F0000309E0000309D0055
:10050800852A141C882A892AA12A18089D071908EF
:1005180003110318013E0319922A9E071A080311B2
:100528000318013E0319992A9F071B080311031892
:10053800013E0319A02AA007A12A01309C0003103C
:10054800980D990D9A0D9B0D9C0BA32A0130031051
:10055800970C960C950C940CFF3E031DAB2A1708BC
:10056800160415041404031DBA2ABB2A852ABC2ABA
:10057800200897001F0896001E0895001D08940083
:10058800C52A0800851530088F002F088E00043012
:1005980003108F0C8E0CFF3E031DCC2A0E088C0016
:1005A8000F088D007F23831285112F08AB003008B8
:1005B800AC00AD01AE010930AF000030B000FF3033
:1005C80081000B111308CF0012088A00110884005B
:1005D800100E8300CE0E4E0E0900D8308312940000
:1005E800723095006A238312051185100510383082
:1005F80086003A309400113095006A23A323BE3058
:1006080083129400053095006A23A3231D308312BA
:100618009400003095006A23A32308301A23013080
:100628001A2306301A230C301A2308008312940068
:100638000511FF308316860083128514232B0510BD
:1006480000008312051400008312861B2C2B2D2B0F
:10065800232B0510831686018312051185101408B3
:100668008600A3230800831294000511FF30831627
:10067800860083128514402B051000008312051490
:1006880000008312861B492B4A2B402B051083162A
:10069800860183120515851014088600A323080017
:1006A80003308A000408840A820700343034313465
:1006B80032343334343435343634373438343934E6
:1006C8004134423443344434453446346C2B6C2B27
:1006D8000130831294020030031C95039502FF3009
:1006E8001506031D792BFF301406031D7C2B7D2B6B
:1006F8006C2B7E2B0800812B812B013083128C02FE
:100708000030031C8D038D02FF300D06031D8E2B58
:10071800FF300C06031D912B922B812B932B080085
:1007280064008001840A0406031900340406952B2A
:1007380083132B3084003930942383011028051447
:060748000000051008008E
:02400E00FEFFB3
:00000001FF
